:020000040000FA
:02000000092ACB
:08000800A000030E8312A10009
:100010002608820020342034203420342034203438
:100020006534733463342E34613473346D34203466
:10003000563431342E3435342034203420342034B6
:100040004534533443344134203420342034203474
:10005000B801B901BA01B90AB601B7010310B50D6B
:10006000B80D03183628B90DBA0D2E28B80CB50CEA
:100070003508B3023808031C013EB402031C4C28A7
:100080003908B6043A08B7040310BA0CB90C0318BF
:100090000800B80CB50C38283508B3070318B40AA3
:1000A0003808B4074428B601B7013508B800381C31
:1000B0005F283308B60734080318013EB70703105A
:1000C000B80C3808031908000310B30DB40D5728F5
:0C00D000313E8200713E8200B13E820091
:1002000085010000062A27088500082200008501D4
:10021000062A2708850005292708850000000B29E4
:10022000270885000E2927088500000012292708C5
:100230008500152927088500000019292708850051
:1002400000001C2927088500042A000085010822D7
:10025000292927088500042A000085010822302961
:100260002729003400340034033409340C341034AA
:10027000133417341A341E34F134F134F134F134B8
:10028000F134F134F134F134F134F134F134F13446
:10029000F134F134F134F134F134F134F134F13436
:1002A000F134F134F134F134F134F134F134F13426
:1002B000F134F134F134F134F134F134F134F13416
:1002C000F134F134F134F134F134F134F134F13406
:1002D000F134F134F134F134F134F1342C34253487
:1002E000223400340034003400340034003400344C
:1002F0000034003400340034FB34FA34F834F7347A
:10030000F534F334F134EF34ED34EB34E934E734DD
:10031000E434E234DF34DC34D934D634D234CF346C
:10032000CB34C734C334BE34B934B434AE34A83457
:10033000A1349A34923489347F34753469345C340E
:100340004D343C3429341334093409340934093424
:1003500009340934093409340934093408340834B7
:100360000834083408340834C834C834C834C834AD
:10037000C834C834C834C834C934C934C934C93499
:10038000C934C934C934C934C934C934C934C93485
:10039000C934C934C934C934C934C934C934C93475
:1003A000C934C934C934C934C934C934C934C93465
:1003B000C934C934C934C934C934C934C934C93455
:1003C000C934C934C934C934CD34D334D934DE3412
:1003D000E434E934EE34F334F834FC3400340034DB
:1003E0000034A218F829A214000085012908FD296B
:1003F000270885002808A210000081000B11210E9B
:100400008300A00E200E09002808FD292908FD29D7
:1004100008008316FF239000831201308A008501B3
:100420008316A83099008312033099008316303068
:10043000023801389F001030950000308100DF3015
:10044000FB3985008312FF3081008B1601309F003D
:10045000A2011430A300A501A701A801A901F13050
:10046000A600FF30AF00B000B100B2008B17DF2252
:100470002218372A4308BC00BE004208BB00403E99
:10048000BD000318BE0ADF222218432A42083D029B
:100490004308031C013E3E020318432A4208BD00E4
:1004A0004308BE003B083D02B300AD003C08031CFE
:1004B000013E3E02B400AE004030B50028203608B0
:1004C000AC00B300B40153203608AD023708031C5A
:1004D000013EAE020310AE0CAD0C3B08AD073C086C
:1004E0000318013EAE07DF222218732A3D0842029C
:1004F0003E08031C013E430203184E2A4208B30083
:100500004308B4000A230038031D732A8B17C52241
:10051000D222C5228B17A501A701B5222308A4006A
:10052000032322188E2A6820003C031D8E2AA40B68
:10053000902A0130A300A7018501A501B522203032
:10054000A700032322188B2A25020319B32A0318B4
:10055000AD2AA50AB5222211A12A221DB12AA5027F
:10056000B5222215A12A2211A12A25086A20AA0053
:1005700025086C20AB00250868208B12A6002A08ED
:10058000A8002B08A9008B160800C830BF00203037
:10059000850008220822082208228501D822BF0BE4
:1005A000C72A0800C830BF00D822BF0BD42A0800D1
:1005B00064003230C0000822C00BDB2A08001E2372
:1005C000221808000530C1000E08C2000F08C30041
:1005D0001E23221808004208FD3EB3004308031CF6
:1005E000FF3EB40033080E02B3003408031C013E82
:1005F0000F02B400031DDF2A073033020318DF2A7D
:10060000C10BE82A08001E23221800340E08B3008C
:100610000F08B4002D08B3022E08031C013EB402DB
:10062000031C00342C08B5002820B708031D3F34F4
:100630004030360203183F3436080800221040309C
:10064000C4001B30C5008E018F01413090004B2348
:10065000221800340E080F040319272B03309F00C3
:100660004B232218003409300F020318452B051EB6
:10067000302B90019F18502B5223553C0318502BC0
:1006800003300F02031C232B08004B2322180034D5
:10069000051E452B232B6400C40B0800C50B080066
:1006A000221408003108B2003008B1002F08B00051
:1006B0001E08AF00C600C7013008C6070318C70AE6
:1006C0003108C6070318C70A3208C6070318C70A45
:0C06D000C70CC60CC70CC60C460808007E
:02400E00CC3FA5
:00000001FF
